:1000000012C01895189518951895189523C118952C
:100010001895189518951895189518951895189578
:100020001895189518958FED8DBFC0ECE0EC4E2E0D
:10003000DD275D2EEEE7F0E0A0E6B0E088278D93A7
:100040003197E9F766248FEF87BB8FEF88BB80E09D
:1000500081BB8FEF82BB82E083BF80E080BF89B726
:10006000826089BF789480E090E0A4E78D939C93B0
:1000700080E080936B008AE080936D00809168003F
:1000800080648093680080E0809376000027A8E673
:100090008C9187FB0EF401E041E0041709F0D7C012
:1000A000809168008F7780936800F1D1ABE68C91E6
:1000B0008F5F8C9340916D0000916B00041781E07D
:1000C00008F480E08F930027A8E68C9186FB0EF45D
:1000D00001E041E0041781E009F080E09F9189236D
:1000E000882309F4B4C080E080936B0088B390E863
:1000F000892788BB00917600003009F010C0A4E782
:10010000EDD2A4E70D911C91043853E0150709F0D6
:1001100005C080E090E0A4E78D939C938ED1009180
:100120007600013009F084C0A4E7D8D2A4E70D918D
:100130001C91023350E0150708F41DC080E090E0E8
:10014000A4E78D939C9383E090E08A939A93CDD219
:100150002296A4E60C9383E090E08A939A93C5D20A
:100160002296A5E60C9383E090E08A939A93BDD201
:100170002296A6E60C9300916400013009F009C0B4
:1001800000916100043608F004C0A1E68C918F5FF5
:100190008C9300916400023009F00CC00091610062
:1001A000003010F009F001C005C08091610081505D
:1001B0008093610000916500013009F009C0009151
:1001C0006300043608F004C0A3E68C918F5F8C9323
:1001D00000916500023009F00CC00091630000300E
:1001E00010F009F001C005C0809163008150809338
:1001F000630000916600013009F009C000916200BF
:10020000043608F004C0A2E68C918F5F8C930091B5
:100210006600023009F00CC000916200003010F05E
:1002200009F001C005C08091620081508093620096
:1002300000917600023009F00AC084E893E08A93C6
:100240009A9353D22296A4E70D931C93F6D01ECF17
:10025000F894FFCF0F921F922F923F924F925F928E
:100260007F92AF92BF920F931F932F933F934F9321
:100270005F936F937F938F939F93AF93BF93CF932E
:10028000DF93EF93FF938FB78F93A0E68C918F5FEF
:100290008C9300916000043609F003C080E08093E5
:1002A00060004091610000916000041708F003C0F5
:1002B000C09AC39A02C0C098C3984091630000914D
:1002C0006000041708F003C0C19AC49A02C0C19824
:1002D000C4984091620000916000041708F003C0C8
:1002E000C29AC59A02C0C298C598A9E6F7D1A9E6F4
:1002F0000D911C910A3F50E0150709F00AC080E0FB
:1003000090E0A9E68D939C9380916800806880932B
:1003100068008F918FBFFF91EF91DF91CF91BF91D7
:10032000AF919F918F917F916F915F914F913F918D
:100330002F911F910F91BF90AF907F905F904F9042
:100340003F902F901F900F901895A0E70D911C9152
:10035000033853E0150710F009F001C00AC0A0E708
:100360000D911C9144E853E0041B150BA0E70D937D
:100370001C93A0E70D911C91043650E0150780E016
:1003800010F009F081E08F93A0E70D911C91043FDC
:1003900051E0150781E008F080E09F9189238823D0
:1003A00009F405C080E090E0A2E78D939C93A0E75C
:1003B0000D911C91043650E0150710F009F00AC0A9
:1003C00004E610E0A0E74D915C91041B150BA2E739
:1003D0000D931C93A0E70D911C91043F51E015076C
:1003E00081E008F480E08F93A0E70D911C9108351F
:1003F00052E0150781E010F009F080E09F91892319
:10040000882309F40AC0A0E70D911C9144EF51E044
:10041000041B150BA2E70D931C93A0E70D911C91F3
:10042000083552E0150710F009F001C005C084E658
:1004300090E0A2E78D939C930895A4E78D919C9101
:10044000A0E78D939C9381DF80917200809361007F
:10045000A4E70D911C914CE251E0040F151FA0E799
:100460000D931C9372DF8091720080936300A4E768
:100470000D911C9148E552E0040F151FA0E70D9364
:100480001C9363DF8091720080936200089500B333
:100490000F3F81E009F480E08F9340B300916F003B
:1004A000041781E009F080E09F918923882309F4F3
:1004B0000EC1AEE68C918F5F8C9300916E000A3076
:1004C00009F004C100916F000E3709F010C085E0FB
:1004D00080936E0000916D00013010F009F001C0B2
:1004E00005C080916D00815080936D00EFC00D3785
:1004F00009F00DC085E080936E0000916D00083218
:1005000008F004C0ADE68C918F5F8C93DFC00C3790
:1005100009F00DC0A8E68C9186FB882780F98095AC
:1005200080FBA8E68C9186F98C93C79ACFC00F36D2
:1005300009F007C08CEB92E0A4E78D939C937DDFDC
:10054000C5C0073709F007C080E991E0A4E78D93A3
:100550009C9373DFBBC00B3709F007C084E690E0C3
:10056000A4E78D939C9369DFB1C00E3609F00DC0EE
:1005700088E080936E0000916100043608F004C0AA
:10058000A1E68C918F5F8C93A1C00D3609F010C04D
:1005900088E080936E0000916100003010F009F057
:1005A00001C005C0809161008150809361008EC0C0
:1005B000063709F00DC088E080936E00009163005B
:1005C000043608F004C0A3E68C918F5F8C937EC044
:1005D000053709F010C088E080936E000091630039
:1005E000003010F009F001C005C080916300815017
:1005F000809363006BC00A3709F00DC088E08093D8
:100600006E0000916200043608F004C0A2E68C91EE
:100610008F5F8C935BC0093709F010C088E080932E
:100620006E0000916200003010F009F001C005C0BA
:100630008091620081508093620048C0073609F0C3
:100640000AC084E68093610084E68093630080E0C2
:10065000809362003BC0033709F00AC080E08093BA
:10066000610084E68093630084E6809362002EC07C
:100670000B3609F00AC084E68093610080E0809325
:10068000630084E68093620021C0033609F00AC04B
:1006900084E68093610084E68093630084E680931F
:1006A000620014C00C3609F004C080E0809376002C
:1006B0000DC0043709F004C081E08093760006C0C5
:1006C000083709F003C082E08093760006C0AFE6E9
:1006D00080B38C9384E080936E000895ED91FC913B
:1006E000EF5FFF4FFC93EE93089540917700509198
:1006F00078000DE815E30BD049E156E3040F151F10
:1007000000937700109378004981588125C008D064
:100710003DD000FC10D0089503D01ED001F8F9CFD1
:100720000024E89457FF02C009D0689400F80BD069
:1007300010F80124089502D009D0089550954095ED
:100740004F5F5F4F0895E89417FF08950095109547
:100750000F5F1F4F68940895352F242FE894452B81
:1007600011F468940895512F402F0027112780E13C
:10077000440F551F001F111F021B130B416018F47B
:10078000020F131F4E7F8A9599F70895752F642FD6
:1007900055274427FF93F1E1889405C010F4460FD4
:1007A000571F5695479517950795FA95B9F7FF91F5
:1007B00008953197F1F70895689462F80895E894E0
:0407C00062F808953E
:00000001FF
